:020000040000FA
:0400000034EF1CF0CD
:040008000BEF1AF0F0
:06002A00D9CFE5FFE1CF94
:10003000D9FF00C0E5FF01C0E5FF02C0E5FF03C036
:10004000E5FF04C0E5FF05C0E5FF06C0E5FF07C00A
:10005000E5FF08C0E5FF040E0101185DD8B09EEF72
:1000600003F009C0E5FF0AC0E5FF0A6A010118357F
:100070000A36E8340A36FC0B096E000EFB6E000EE1
:10008000FA6E9A0E09260A50FA22D8B0FB2A0950B5
:10009000E4CF0AF0E4CF09F0F96E55EF00F031EF4C
:1000A00001F01AEF02F048EF03F0000E016EA00E0F
:1000B000006E800E026E000EE56E200EE56E340EB0
:1000C000E56E0250E56E0150E56E0050E56EE3EC22
:1000D00013F0060EE126000E016EA10E006E800EDA
:1000E000026E0001F451E56E0001F351E56E020E5F
:1000F000E56E0250E56E0150E56E0050E56E35ECA0
:1001000008F0060EE126300E01011925006E0050A0
:100110000001A96F000E016EAC0E006E800E026E23
:100120000001BB51036E0001BC51046E056A066AF2
:10013000000EE56E000EE56E000EE56E0A0EE56E31
:100140000650E56E0550E56E0450E56E0350E56E11
:100150007AEC10F0036EF3CF04F0F4CF05F0E9CFA2
:1001600006F0080EE1260350E56E0250E56E0150E0
:10017000E56E0050E56EE4EC0CF0040EE126000E96
:10018000016EA00E006E800E026E0250E56E0150F0
:10019000E56E0050E56E000EE56E000EE56E8FEC2C
:1001A00012F0050EE126000E016EA00E006E800E0C
:1001B000026E000EE56E200EE56E460EE56E0250F4
:1001C000E56E0150E56E0050E56EE3EC13F0060EAF
:1001D000E126000E016EA10E006E800E026EF1C0CF
:1001E00003F0F2C004F00450E56E0350E56E020E19
:1001F000E56E0250E56E0150E56E0050E56E35EC9F
:1002000008F0060EE126000E016EA90E006E800EAB
:10021000026E0001F651E56E0001F551E56E020E29
:10022000E56E0250E56E0150E56E0050E56E35EC6E
:1002300008F0060EE126000E016EA00E006E800E84
:10024000026E0250E56E0150E56E0050E56E010E43
:10025000E56E000EE56E8FEC12F0050EE1269EEFC6
:1002600003F0000EE56E640EE56E0001F851E56ED8
:100270000001F751E56E66EC15F0006EF3CF01F06A
:10028000040EE126000EE56E640EE56E0001F251EB
:10029000E56E0001F151E56E14EC12F0026EF3CF41
:1002A00003F0040EE1260350E56E0250E56E0150A6
:1002B000E56E0050E56E61EC16F0006EF3CF01F0D4
:1002C000040EE126000E036EA00E026E800E046E78
:1002D000000EE56E200EE56E580EE56E0450E56EDC
:1002E0000350E56E0250E56EE3EC13F0060EE126D6
:1002F000000E036EA10E026E800E046E0001F85116
:10030000E56E0001F751E56E020EE56E0450E56EF4
:100310000350E56E0250E56E35EC08F0060EE1265E
:10032000000E036EA90E026E800E046EF1C005F081
:10033000F2C006F00650E56E0550E56E020EE56E61
:100340000450E56E0350E56E0250E56E35EC08F0A2
:10035000060EE126000E036EA00E026E800E046EE5
:100360000450E56E0350E56E0250E56E000EE56E3A
:10037000000EE56E8FEC12F0050EE126000E036E06
:10038000A00E026E800E046E000EE56E200EE56E6D
:100390006A0EE56E0450E56E0350E56E0250E56EA0
:1003A000E3EC13F0060EE126000E036EA20E026EC1
:1003B000800E046E0150E56E0050E56E000EE56E95
:1003C0000450E56E0350E56E0250E56E35EC08F022
:1003D000060EE126000E036EAA0E026E800E046E5B
:1003E000BFEC17F0056EF3CF06F00650E56E055032
:1003F000E56E000EE56E0450E56E0350E56E0250AA
:10040000E56E35EC08F0060EE126000E036EA00E38
:10041000026E800E046E0450E56E0350E56E0250CD
:10042000E56E010EE56E000EE56E8FEC12F0050E26
:10043000E12684D1000E036EA00E026E800E046EC3
:10044000000EE56E200EE56E7C0EE56E0450E56E46
:100450000350E56E0250E56EE3EC13F0060EE12664
:100460000001F9510001FA11D8B477D0000E036EE3
:10047000A10E026E800E046EF9C005F0FAC006F0FF
:10048000076A086A0850E56E0750E56E0650E56E8B
:100490000550E56E0001C051E56E0001BF51E56EEB
:1004A0000001BE51E56E0001BD51E56E7AEC10F021
:1004B000056EF3CF06F0F4CF07F0E9CF08F0080E91
:1004C000E1260650E56E0550E56E020EE56E04501D
:1004D000E56E0350E56E0250E56E35EC08F0060E51
:1004E000E126000E036EA90E026E800E046EF9C0A6
:1004F00005F0FAC006F0076A086A0850E56E075072
:10050000E56E0650E56E0550E56E0001C451E56EDE
:100510000001C351E56E0001C251E56E0001C151F9
:10052000E56E7AEC10F0056EF3CF06F0F4CF07F02D
:10053000E9CF08F0080EE1260650E56E0550E56E9D
:10054000020EE56E0450E56E0350E56E0250E56E56
:1005500035EC08F0060EE1262CD0000E036EA10E3D
:10056000026E800E046E000EE56E000EE56E020E49
:10057000E56E0450E56E0350E56E0250E56E35EC15
:1005800008F0060EE126000E036EA90E026E800E24
:10059000046E000EE56E000EE56E020EE56E045070
:1005A000E56E0350E56E0250E56E35EC08F0060E80
:1005B000E126000E036EA00E026E800E046E045043
:1005C000E56E0350E56E0250E56E000EE56E000E1E
:1005D000E56E8FEC12F0050EE126000E036EA00E04
:1005E000026E800E046E000EE56E200EE56E8E0E1D
:1005F000E56E0450E56E0350E56E0250E56EE3ECE7
:1006000013F0060EE126000E036EA10E026E800EA0
:10061000046E0001FC51E56E0001FB51E56E020E17
:10062000E56E0450E56E0350E56E0250E56E35EC64
:1006300008F0060EE126000E036EA90E026E800E73
:10064000046E0001FE51E56E0001FD51E56E020EE3
:10065000E56E0450E56E0350E56E0250E56E35EC34
:1006600008F0060EE126000E036EA00E026E800E4C
:10067000046E0450E56E0350E56E0250E56E010E07
:10068000E56E000EE56E8FEC12F0050EE12656D0F9
:10069000000EE56E200EE56EA00EE56E000EE56E16
:1006A000000EE56E8FEC12F0050EE126000E036ED3
:1006B000A00E026E800E046E000EE56E200EE56E3A
:1006C000B20EE56E0450E56E0350E56E0250E56E25
:1006D000E3EC13F0060EE1260C0EE56EF0EC18F0DC
:1006E000006EF3CF01F0E12A000E036EAB0E026E36
:1006F000800E046E0150E56E0050E56E000EE56E52
:100700000450E56E0350E56E0250E56E35EC08F0DE
:10071000060EE126000E016EA00E006E800E026E27
:100720000250E56E0150E56E0050E56E010EE56E7B
:10073000000EE56E8FEC12F0050EE126E4CF08F016
:10074000E4CF07F0E4CF06F0E4CF05F0E4CF04F007
:10075000E4CF03F0E4CF02F0E4CF01F0E4CF00F007
:10076000E4CFD9FF1200D36AFF0E926E0F0E936E84
:10077000FF0E946E816A010E01011B6F0101186B5F
:10078000060EE56EF0EC18F00101066FF3CF07F1ED
:10079000E12A080EE56EF0EC18F00101086FF3CFC6
:1007A00009F1E12A0001F36B0001F46B01010A6B0E
:1007B00001010B6B0001C56B0001C66B0001C76B2B
:1007C0000001C86B0001F56B0001F66B0101026BC3
:1007D0000101036B0101046B0101056B81800101C3
:1007E000006B0101016B01011A6B0101106B01012A
:1007F000116B01011C6B01011D6B0001FB6B000102
:10080000FC6B0001FD6B0001FE6B0001BD6B000184
:10081000BE6B0001BF6B0001C06B0001C16B00012A
:10082000C26B0001C36B0001C46B0001F96B0001D6
:10083000FA6B006A82B0002A00C019F10101195157
:1008400011E008C100F009C101F0026A036A015019
:100850000001BC6F00500001BB6F0001B96B0001CB
:10086000BA6B10D006C100F007C101F0026A036A3A
:1008700001500001BC6F00500001BB6F0001B96B5B
:100880000001BA6B74EC1BF078EC18F05FEC1BF015
:10089000C0EC1BF0DEEC1BF0D0A602D0A2EC1AF0EC
:1008A000D18015EC00F0F26AF28CA082F18CF28813
:1008B000F28EEBEC1BF0A00E0001CD6F860E000156
:1008C000CE6F010E0001CF6F0001D06B006A81B8BE
:1008D000002A0050D880E866D890006A00360050A0
:1008E000010BE838F46E8150EF0BF410816E006A52
:1008F00082B0002A19C101F00150001801E15DD059
:10090000010119512BE00001BB51006E0001BC51E7
:10091000016E026A036A00500101086F0150010173
:10092000096F01010951E56E01010851E56E080EDC
:10093000E56EB5EC18F0030EE12606C100F007C124
:1009400001F0026A036A01500001BC6F005000010F
:10095000BB6F0001B96B0001BA6B2AD00001BB511B
:10096000006E0001BC51016E026A036A0050010171
:10097000066F01500101076F01010751E56E01018A
:100980000651E56E060EE56EB5EC18F0030EE12695
:1009900008C100F009C101F0026A036A01500001B8
:1009A000BC6F00500001BB6F0001B96B0001BA6B56
:1009B000006A82B0002A00C019F1000EE56E40EC1A
:1009C0001AF0006EF3CF01F0E12A0150E56E0050FD
:1009D000E56E000EE56E260EE56E61EC16F0006E1B
:1009E000F3CF01F0040EE126000EE56E0B0EE56E6E
:1009F0000150E56E0050E56E66EC15F00001F76FF2
:100A0000F3CFF8F0040EE12601011051010111119C
:100A100015E1070E0001F85D03E1D10E0001F75D5D
:100A200007E3340E0101106F080E0101116F06D0AB
:100A30001A0E0101106F040E0101116F006A0A0EF7
:100A4000005CD8B0EFD0D5EC19F0016EF3CF02F016
:100A5000F4CF03F0E9CF04F00001D051045C0BE1C6
:100A60000001CF51035C07E10001CE51025C03E1BC
:100A70000001CD51015CE7E3A00E0001CD27860EF9
:100A80000001CE23010E0001CF23000E0001D02370
:100A9000010EE56E40EC1AF0016EF3CF02F0E12A90
:100AA0000C0E0126FE0E0222020E025C02E1000E76
:100AB000015C02E3016A026A0250E56E0150E56ED4
:100AC000000EE56E790EE56E61EC16F0016EF3CF67
:100AD00002F0040EE126000EE56E060EE56E0250F1
:100AE000E56E0150E56E66EC15F00001F16FF3CF95
:100AF000F2F0040EE126010111510001F85D04E15C
:100B0000010110510001F75D0EE201011A8101019E
:100B10001C2B290E01011C5D0DE3140E01011D6F3C
:100B200001011C6B07D001011D5104E101011A9163
:100B300001011C6B39EC0EF00050010A03E15EEC80
:100B40000FF06ED00050020A03E115EC1BF068D0E4
:100B50000050030A03E105EC13F062D00050040AD0
:100B600003E177EC13F05CD00050050A01E04DD0B2
:100B70000C0EE56EF0EC18F0016EF3CF02F0E12AF6
:100B8000000EE56E0F0EE56E420EE56E400EE56E50
:100B90000001D051E56E0001CF51E56E0001CE514C
:100BA000E56E0001CD51E56E7AEC10F0026EF3CFE8
:100BB00003F0F4CF04F0E9CF05F0080EE126066A51
:100BC000076A086A0850E56E0750E56E0650E56E44
:100BD0000150E56E0550E56E0450E56E0350E56E7C
:100BE0000250E56ECCEC0EF0016EF3CF02F0F4CFC4
:100BF00003F0E9CF04F0080EE126015002100310C3
:100C000004100EE107EC11F00BD00050060A03E1CE
:100C100040EC17F005D00050090A02E115EC00F095
:100C2000002A0DD7010119511BE00001BB51006ED4
:100C30000001BC51016E026A036A00500101086F95
:100C400001500101096F01010951E56E01010851CF
:100C5000E56E080EE56EB5EC18F0030EE1261AD02D
:100C60000001BB51006E0001BC51016E026A036AB3
:100C700000500101066F01500101076F010107518A
:100C8000E56E01010651E56E060EE56EB5EC18F055
:100C9000030EE1260D0E0001F45D03E1490E000193
:100CA000F35DD8A036D00001F251800F7C0F03E134
:100CB000B10E0001F15D2DE3F3C000F0F4C001F0CE
:100CC000026A036A00500001BD2701500001BE23E3
:100CD00002500001BF2303500001C023F1C000F007
:100CE000F2C001F0E86A0001F2BFFF0E026E036E6F
:100CF00000500001C12701500001C2230250000131
:100D0000C32303500001C4230001F92B02E30001B7
:100D1000FA2B040066EF04F01200D9CFE5FFE1CF13
:100D2000D9FF00C0E5FF01C0E5FF02C0E5FF03C039
:100D3000E5FF04C0E5FF05C0E5FF000E016E800E73
:100D4000006E800E026E030EE56E0250E56E0150DD
:100D5000E56E0050E56E000EE56E000EE56E000ECD
:100D6000E56ED00EE56E9AEC0DF0080EE126000E51
:100D7000016E830E006E800E026E030EE56E025051
:100D8000E56E0150E56E0050E56E000EE56E000E5A
:100D9000E56E040EE56ED00EE56E9AEC0DF0080ED1
:100DA000E126000E016E860E006E800E026E0001BE
:100DB000F751036E03C0E5FF00C0E9FF01C0F3FF78
:100DC00002504AEC1CF0002AD8B0012AD8B0022AFE
:100DD0000001F851036E046A03C0E5FF00C0E9FF9B
:100DE00001C0F3FF02504AEC1CF0002AD8B0012ADF
:100DF000D8B0022A0001F151036E03C0E5FF00C024
:100E0000E9FF01C0F3FF02504AEC1CF0002AD8B001
:100E1000012AD8B0022A0001F251036E046A03BE0F
:100E2000046803C0E5FF00C0E9FF01C0F3FF025002
:100E30004AEC1CF0002AD8B0012AD8B0022A0101DD
:100E40000651036E03C0E5FF00C0E9FF01C0F3FFD8
:100E500002504AEC1CF0002AD8B0012AD8B0022A6D
:100E600001010751036E046A03C0E5FF00C0E9FFFA
:100E700001C0F3FF02504AEC1CF0002AD8B0012A4E
:100E8000D8B0022A01010851036E03C0E5FF00C07B
:100E9000E9FF01C0F3FF02504AEC1CF0002AD8B071
:100EA000012AD8B0022A01010951036E046A03C065
:100EB000E5FF00C0E9FF01C0F3FF02504AEC1CF05F
:100EC000002AD8B0012AD8B0022A0001F351036EDB
:100ED00003C0E5FF00C0E9FF01C0F3FF02504AEC88
:100EE0001CF0002AD8B0012AD8B0022A0001F4511F
:100EF000036E046A03C0E5FF00C0E9FF01C0F3FF11
:100F000002504AEC1CF0002AD8B0012AD8B0022ABC
:100F10000001F551036E03C0E5FF00C0E9FF01C009
:100F2000F3FF02504AEC1CF0002AD8B0012AD8B0D6
:100F3000022A0001F651036E046A03C0E5FF00C0F7
:100F4000E9FF01C0F3FF02504AEC1CF0002AD8B0C0
:100F5000012AD8B0022A000EE56E00C0E9FF01C0E8
:100F6000F3FF02504AEC1CF0002AD8B0012AD8B096
:100F7000022A000EE56E00C0E9FF01C0F3FF025037
:100F80004AEC1CF0002AD8B0012AD8B0022A01018C
:100F90000A51036E03C0E5FF00C0E9FF01C0F3FF83
:100FA00002504AEC1CF0002AD8B0012AD8B0022A1C
:100FB00019C1E5FF00C0E9FF01C0F3FF02504AEC90
:100FC0001CF0002AD8B0012AD8B0022A000EE56E23
:100FD00000C0E9FF01C0F3FF02504AEC1CF0002AF8
:100FE000D8B0012AD8B0022A000EE56E00C0E9FF91
:100FF00001C0F3FF02504AEC1CF0002AD8B0012ACD
:10100000D8B0022A0A0EE56EF0EC18F0036EF3CFAA
:1010100004F0E12A0350056E05C0E5FF00C0E9FFBA
:1010200001C0F3FF02504AEC1CF0002AD8B0012A9C
:10103000D8B0022A0450036E046A03C0E5FF00C062
:10104000E9FF01C0F3FF02504AEC1CF0E4CF05F0C9
:10105000E4CF04F0E4CF03F0E4CF02F0E4CF01F0FA
:10106000E4CF00F0E4CFD9FF1200D9CFE5FFE1CF04
:10107000D9FF00C0E5FF01C0E5FF02C0E5FF03C0E6
:10108000E5FF04C0E5FF05C0E5FF06C0E5FF07C0BA
:10109000E5FF08C0E5FF09C0E5FF0AC0E5FF020E55
:1010A000DBCF00F0030EDBCF01F0040EDBCF02F04C
:1010B000050EDBCF03F0060EDBCF04F0070EDBCF0F
:1010C00005F000C006F001C007F002C008F00350B0
:1010D00003E003500508036E270EE56E100EE56E63
:1010E0000550E56E0450E56E66EC15F0096EF3CF21
:1010F0000AF0040EE126300E092609C0E5FF06C0FD
:10110000E9FF07C0F3FF08504AEC1CF0062AD8B0EC
:10111000072AD8B0082A030603500EE12E0EE56E0A
:1011200006C0E9FF07C0F3FF08504AEC1CF0062A8E
:10113000D8B0072AD8B0082A270EE56E100EE56E43
:101140000550E56E0450E56EB1EC14F0046EF3CF7B
:1011500005F0040EE126030EE56EE80EE56E05507F
:10116000E56E0450E56E66EC15F0096EF3CF0AF0FB
:10117000040EE126300E092609C0E5FF06C0E9FF8E
:1011800007C0F3FF08504AEC1CF0062AD8B0072A23
:10119000D8B0082A030603500EE12E0EE56E06C0F5
:1011A000E9FF07C0F3FF08504AEC1CF0062AD8B04C
:1011B000072AD8B0082A030EE56EE80EE56E055042
:1011C000E56E0450E56EB1EC14F0046EF3CF05F05B
:1011D000040EE126000EE56E640EE56E0550E56E28
:1011E0000450E56E66EC15F0096EF3CF0AF0040EBC
:1011F000E126300E092609C0E5FF06C0E9FF07C059
:10120000F3FF08504AEC1CF0062AD8B0072AD8B0E1
:10121000082A030603500EE12E0EE56E06C0E9FF14
:1012200007C0F3FF08504AEC1CF0062AD8B0072A82
:10123000D8B0082A000EE56E640EE56E0550E56E26
:101240000450E56EB1EC14F0046EF3CF05F0040E1B
:10125000E126000EE56E0A0EE56E0550E56E0450BF
:10126000E56E66EC15F0096EF3CF0AF0040EE12688
:10127000300E092609C0E5FF06C0E9FF07C0F3FFED
:1012800008504AEC1CF0062AD8B0072AD8B0082A21
:10129000030603500EE12E0EE56E06C0E9FF07C0FF
:1012A000F3FF08504AEC1CF0062AD8B0072AD8B041
:1012B000082A000EE56E0A0EE56E0550E56E045034
:1012C000E56EB1EC14F0046EF3CF05F0040EE126E8
:1012D000300E042604C0E5FF06C0E9FF07C0F3FF97
:1012E00008504AEC1CF0062AD8B0072AD8B0082AC1
:1012F000032E09D02E0EE56E06C0E9FF07C0F3FFEE
:1013000008504AEC1CF00050040F036E000E012040
:10131000046E000E0220056E0250800FF36E055021
:10132000800FF35C05E10450015C02E10350005CB6
:101330001AE200C0E9FF01C0F3FF0250AFEC1BF05E
:10134000066E0650300A0FE1200EE56E00C0E9FF80
:1013500001C0F3FF02504AEC1CF0002AD8B0012A69
:10136000D8B0022AD9D7E4CF0AF0E4CF09F0E4CF0D
:1013700008F0E4CF07F0E4CF06F0E4CF05F0E4CFC7
:1013800004F0E4CF03F0E4CF02F0E4CF01F0E4CFC7
:1013900000F0E4CFD9FF1200D9CFE5FFE1CFD9FFAC
:1013A00000C0E5FF01C0E5FF02C0E5FF03C0E5FFA7
:1013B00004C0E5FF05C0E5FF06C0E5FF000E016EB5
:1013C000C90E006E800E026E640EE56E9DEC1BF081
:1013D000E12A40EC1CF0036E03C0E5FF00C0E9FF0A
:1013E00001C0F3FF02504AEC1CF0002AD8B0012AD9
:1013F000D8B0022A40EC1CF0036E03C0E5FF00C029
:10140000E9FF01C0F3FF02504AEC1CF0002AD8B0FB
:10141000012AD8B0022A40EC1CF0036E03C0E5FF9D
:1014200000C0E9FF01C0F3FF02504AEC1CF0002AA3
:10143000D8B0012AD8B0022A40EC1CF0036E03C0D9
:10144000E5FF00C0E9FF01C0F3FF02504AEC1CF0C9
:10145000010E016E0C0E006E800E026E00C003F0D5
:1014600001C004F002C005F040EC1CF0066E06C09E
:10147000E5FF03C0E9FF04C0F3FF05504AEC1CF090
:10148000002AD8B0012AD8B0022A40EC1CF0036E22
:1014900003C0E5FF00C0E9FF01C0F3FF02504AECC2
:1014A0001CF0006A016A01010D51015C03E10101B8
:1014B0000C51005CD8B093D040EC1CF0026E02508E
:1014C000720A01E18CD00001CC51E56E0001CB51D4
:1014D000E56E0001CA51E56E0001C951E56E000ECE
:1014E000E56E000EE56E000EE56E200EE56E00EC7A
:1014F0000BF0026EF3CF03F0F4CF04F0E9CF05F068
:10150000080EE126000E056E800E046E800E066E3B
:10151000200EE56E0650E56E0550E56E0450E56E52
:10152000030EE56E0350E56E0250E56EA00EE56E0B
:101530009AEC0DF0080EE126020EE56E000EE56E47
:10154000200EE56ED60EE56EFDEC16F0040EE126DB
:10155000000E036E800E026E800E046E200EE56E8D
:101560000450E56E0350E56E0250E56EFDEC16F09A
:10157000040EE126C9C002F0CAC003F0CBC004F0DB
:10158000CCC005F00250010F0001C96F000E03200E
:101590000001CA6F000E04200001CB6F000E052071
:1015A0000001CC6F000E0001CC5D0BE1000E0001CC
:1015B000CB5D07E1040E0001CA5D03E1000E0001EE
:1015C000C95D08E30001C96B0001CA6B0001CB6B68
:1015D0000001CC6B0400002AD8B0012A64D7E4CF04
:1015E00006F0E4CF05F0E4CF04F0E4CF03F0E4CF5D
:1015F00002F0E4CF01F0E4CF00F0E4CFD9FF120015
:10160000D9CFE5FFE1CFD9FF00C0E5FF01C0E5FF7D
:1016100002C0E5FF03C0E5FF04C0E5FF05C0E5FF2C
:1016200006C0E5FF07C0E5FF020EDBCF00F0030EAA
:10163000DBCF01F0040EDBCF02F0050EDBCF03F0B1
:10164000060EDBCF04F0070EDBCF05F0080EDBCF74
:1016500006F0090EDBCF07F000500001D16F0150FA
:10166000D26F0250D36F0350D46F04500001D56F76
:101670000550D66F0650D76F0750D86F0001D15173
:101680000001D703F3CF00F0F4CF01F000500001C8
:10169000DB6F0150DC6F0001D1510001D503F3CFA6
:1016A00000F0F4CF01F000500001D96F0150DA6F63
:1016B0000001D4510001D503F3CF00F00001DC514B
:1016C00000260050DC6F0001D3510001D603F3CF98
:1016D00000F00001DC5100260050DC6F0001D35106
:1016E0000001D503F3CF00F0F4CF01F00001DB518E
:1016F0000026DC5101220050DB6F0150DC6F00013D
:10170000D2510001D603F3CF00F0F4CF01F0000175
:10171000DB510026DC5101220050DB6F0150DC6FF1
:101720000001D2510001D703F3CF00F000500001B7
:10173000E06F0001D2510001D503F3CF00F0F4CFE8
:1017400001F000500001DE6F0150DF6F0001D15148
:101750000001D803F3CF00F000500001E46F000156
:10176000D1510001D603F3CF00F0F4CF01F00050C7
:101770000001E26F0150E36F0001DD6B0001E16BDE
:101780000001DD510001D925006E0001DE5100018C
:10179000DA21016E0001DF510001DB21026E000140
:1017A000E0510001DC21036E0050D96F0150DA6F67
:1017B0000250DB6F0350DC6F0001E1510001D925BD
:1017C000006E0001E2510001DA21016E0001E351D7
:1017D0000001DB21026E0001E4510001DC21036EF7
:1017E00003C0E9FF02C0F4FF01C0F3FF0050E4CFE3
:1017F00007F0E4CF06F0E4CF05F0E4CF04F0E4CF47
:1018000003F0E4CF02F0E4CF01F0E4CF00F0E4CF46
:10181000D9FF1200D9CFE5FFE1CFD9FF00C0E5FF26
:1018200001C0E5FF02C0E5FF03C0E5FF000E016E49
:10183000B10E006E800E026E740EE56E9DEC1BF014
:10184000E12A040040EC1CF0036E03C0E5FF00C079
:10185000E9FF01C0F3FF02504AEC1CF0002AD8B0A7
:10186000012AD8B0022A740EE56E9DEC1BF0E12A25
:1018700040EC1CF0036E03C0E5FF00C0E9FF01C0AF
:10188000F3FF02504AEC1CF0002AD8B0012AD8B06D
:10189000022A740EE56E9DEC1BF0E12A40EC1CF070
:1018A000036E03C0E5FF00C0E9FF01C0F3FF025073
:1018B0004AEC1CF0002AD8B0012AD8B0022A740ED3
:1018C000E56E9DEC1BF0E12A030EE56E00C0E9FF1A
:1018D00001C0F3FF02504AEC1CF0002AD8B0012AE4
:1018E000D8B0022A040040EC1CF0036E03C0E5FFF0
:1018F00000C0E9FF01C0F3FF02504AEC1CF0002ACF
:10190000D8B0012AD8B0022A740EE56E9DEC1BF007
:10191000E12A40EC1CF0036E03C0E5FF00C0E9FFC4
:1019200001C0F3FF02504AEC1CF0002AD8B0012A93
:10193000D8B0022A740EE56E9DEC1BF0E12A40EC53
:101940001CF0036E03C0E5FF00C0E9FF01C0F3FF18
:1019500002504AEC1CF0002AD8B0012AD8B0022A62
:10196000740EE56E9DEC1BF0E12A100EE56E00C0D2
:10197000E9FF01C0F3FF02504AEC1CF00400000E26
:10198000016EB10E006E800E026E080EE56E025002
:10199000E56E0150E56E0050E56E000EE56E000E3E
:1019A000E56E000EE56ED00EE56E93EC11F0080EBC
:1019B000E126E4CF03F0E4CF02F0E4CF01F0E4CF7E
:1019C00000F0E4CFD9FF1200D9CFE5FFE1CFD9FF76
:1019D00000C0E5FF01C0E5FF02C0E5FF03C0E5FF71
:1019E00004C0E5FF05C0E5FF06C0E5FF07C0E5FF51
:1019F000020EDBCF00F0030EDBCF01F0040EDBCFD5
:101A000002F0050EDBCF03F0640EE56E03C0E5FFC8
:101A10009EEC19F0046EE450E450300E042604C02D
:101A2000E5FF00C0E9FF01C0F3FF02504AEC1CF0E3
:101A30000050010F046E000E0120056E000E022002
:101A4000066E640EE56E03C0E5FF64EC19F0036EEC
:101A5000E450E4500A0EE56E03C0E5FF9EEC19F079
:101A6000076EE450E450300E072607C0E5FF04C0BF
:101A7000E9FF05C0F3FF06504AEC1CF0042AD8B079
:101A8000052AD8B0062A0A0EE56E03C0E5FF64EC0D
:101A900019F0036EE450E450300E032603C0E5FF56
:101AA00004C0E9FF05C0F3FF06504AEC1CF00050EB
:101AB000020F036E000E0120046E000E0220056E60
:101AC0000250800FF36E0550800FF35C05E1045067
:101AD000015C02E10350005C1AE200C0E9FF01C0B2
:101AE000F3FF0250AFEC1BF0066E0650300A0FE118
:101AF000200EE56E00C0E9FF01C0F3FF02504AEC82
:101B00001CF0002AD8B0012AD8B0022AD9D7E4CFD5
:101B100007F0E4CF06F0E4CF05F0E4CF04F0E4CF23
:101B200003F0E4CF02F0E4CF01F0E4CF00F0E4CF23
:101B3000D9FF1200D9CFE5FFE1CFD9FF00C0E5FF03
:101B400001C0E5FF02C0E5FF03C0E5FF04C0E5FFFB
:101B500005C0E5FF06C0E5FF07C0E5FF08C0E5FFDB
:101B6000020EDBCF00F0030EDBCF01F0040EDBCF63
:101B700002F0050EDBCF03F0060EDBCF04F0070EFC
:101B8000DBCF05F0080EDBCF06F0090EDBCF07F048
:101B900073EC1AF003A003D0020EC86E02D0090E37
:101BA000C86E28EC1CF00050E56E04EC1CF0E12A35
:101BB00003A208D00250036E086A0350E56E04ECDD
:101BC0001CF0E12A0150E56E04EC1CF0E12A1CEC4B
:101BD0001CF000800050E56E04EC1CF0E12A04C00B
:101BE00000F005C001F006C002F007C003F0020ECD
:101BF000035C16E3010EE56EF3EC1AF0046EE12AC5
:101C000004C0E5FF00C0E9FF01C0F3FF02504AEC49
:101C10001CF0002AD8B0012AD8B0022A0306E7D760
:101C200003500FE0000EE56EF3EC1AF0036EE12AAC
:101C300003C0E5FF00C0E9FF01C0F3FF02504AEC1A
:101C40001CF010EC1CF0E86AE4CF08F0E4CF07F0D9
:101C5000E4CF06F0E4CF05F0E4CF04F0E4CF03F0E6
:101C6000E4CF02F0E4CF01F0E4CF00F0E4CFD9FFFD
:101C70001200D9CFE5FFE1CFD9FF00C0E5FF01C0D9
:101C8000E5FF02C0E5FF090EE56E40EC1AF0006EBC
:101C9000F3CF01F0E12A200E0026D8B0012A003649
:101CA0000136003601360034030B0118011A011801
:101CB000006E0050D8B463D000C001F0026A015039
:101CC00001010E1905E1025001010F1901E157D080
:101CD00000500A0A03E10DEC15F051D00050010A42
:101CE0000AE10101182B040E0101185DD8A047D0AC
:101CF0000101186B44D00050020A1BE10101185188
:101D0000030A01E03CD00C0EE56EF0EC18F0016E19
:101D1000F3CF02F0E12A012AD8B0022A0250E56E80
:101D20000150E56E0C0EE56EB5EC18F0030EE126E1
:101D300026D00050040A23E101011851030A1FE1D3
:101D40000C0EE56EF0EC18F0016EF3CF02F0E12A14
:101D5000FF0E0126D8A00206000E025C02E1010E71
:101D6000015C03E2010E016E026A0250E56E015051
:101D7000E56E0C0EE56EB5EC18F0030EE12600C022
:101D80000EF101010F6BE4CF02F0E4CF01F0E4CFDC
:101D900000F0E4CFD9FF1200D9CFE5FFE1CFD9FFA2
:101DA00000C0E5FF01C0E5FF02C0E5FF03C0E5FF9D
:101DB00004C0E5FF05C0E5FF06C0E5FF07C0E5FF7D
:101DC00008C0E5FF09C0E5FF0AC0E5FF020EDBCF52
:101DD00000F0030EDBCF01F0040EDBCF02F0050EA6
:101DE000DBCF03F0060EDBCF04F0070EDBCF05F0F0
:101DF000080EDBCF06F0090EDBCF07F0086A096A90
:101E00000744010B0A6E0AB01BD0045004260536A5
:101E1000063607360750035C08E10650025C05E110
:101E20000550015C02E10450005C06E2D8900732E4
:101E300006320532043204D0092A09C008F0E0D77E
:101E40000750035C08E10650025C05E10550015CA7
:101E500002E10450005C08E30450005E0550015AA2
:101E60000650025A0750035AD890073206320532FC
:101E7000043208C009F008060950E2E103C0E9FF96
:101E800002C0F4FF01C0F3FF0050E4CF0AF0E4CF3A
:101E900009F0E4CF08F0E4CF07F0E4CF06F0E4CF98
:101EA00005F0E4CF04F0E4CF03F0E4CF02F0E4CF98
:101EB00001F0E4CF00F0E4CFD9FF1200D9CFE5FF65
:101EC000E1CFD9FF00C0E5FF01C0E5FF02C0E5FF9B
:101ED00003C0E5FF0101025101010311D8B44AD04A
:101EE000010104510101005D006E01010551010174
:101EF0000159016E000EE56E0A0EE56E0150E56EA9
:101F00000050E56E66EC15F0006EF3CF01F0040EA4
:101F1000E12601010351E56E01010251E56E050E56
:101F2000E56EB40EE56E61EC16F0026EF3CF03F0D1
:101F3000040EE1260150E56E0050E56E0350E56E9B
:101F40000250E56E66EC15F0006EF3CF01F0040E62
:101F5000E1260150E56E0050E56E000EE56E240EA0
:101F6000E56E61EC16F00001F36FF3CFF4F0040EB0
:101F7000E12604D00001F36B0001F46B0001F45181
:101F80000001FC5D04E10001F3510001FB5D11E281
:101F90000001F251800F7C0F03E1B10E0001F15DF1
:101FA00008E3F3C0FBF0F4C0FCF0F1C0FDF0F2C0B8
:101FB000FEF00101026B0101036B00C104F101C1DC
:101FC00005F1E4CF03F0E4CF02F0E4CF01F0E4CF79
:101FD00000F0E4CFD9FF1200D9CFE5FFE1CFD9FF60
:101FE00000C0E5FF01C0E5FF02C0E5FF03C0E5FF5B
:101FF000020EDBCF00F0030EDBCF01F000C002F0D9
:1020000001C003F0FF0E0026D8A001060250031005
:1020100006E0FA0E026E0000022EFDD7EFD7E4CFE5
:1020200003F0E4CF02F0E4CF01F0E4CF00F0E4CF1E
:10203000D9FF1200532020202020202042202020E1
:10204000202020250000492020202020202044207E
:10205000202020202020000056202020202020208A
:102060004920202020202020000050202020202057
:102070002020542020202020202000005341202018
:1020800020202020494120202020202000005350E3
:102090002020202020204950202020202020000027
:1020A000506172616D6574657220536574202020E3
:1020B00000004C6F675365636F6E647320202020AF
:1020C0002020000042617474657279204C6F772083
:1020D0002020202000004141000043617220580070
:1020E000526561647920746F20526F6C6C202E2EC3
:1020F0002E2E0000D9CFE5FFE1CFD9FF00C0E5FFCC
:1021000001C0E5FF02C0E5FF03C0E5FF04C0E5FF35
:1021100005C0E5FF06C0E5FF07C0E5FF08C0E5FF15
:1021200009C0E5FF0AC0E5FF0BC0E5FF0CC0E5FFF5
:102130000DC0E5FF020EDBCF00F0030EDBCF01F098
:10214000040EDBCF02F0050EDBCF03F0060EDBCF73
:1021500004F0070EDBCF05F0080EDBCF06F0090E0A
:10216000DBCF07F0086A096A0A6A0B6A200E0C6E58
:102170000344010B0D6E010E0D16005000260136B2
:10218000023603360850082609360A360B360D503B
:10219000D8A4088007500B5C08E106500A5C05E1F2
:1021A0000550095C02E10450085C09E30450085E34
:1021B0000550095A06500A5A07500B5A00800C2E37
:1021C000D7D703C0E9FF02C0F4FF01C0F3FF0050FE
:1021D000E4CF0DF0E4CF0CF0E4CF0BF0E4CF0AF045
:1021E000E4CF09F0E4CF08F0E4CF07F0E4CF06F045
:1021F000E4CF05F0E4CF04F0E4CF03F0E4CF02F045
:10220000E4CF01F0E4CF00F0E4CFD9FF1200D9CF42
:10221000E5FFE1CFD9FF00C0E5FF01C0E5FF02C047
:10222000E5FF03C0E5FF04C0E5FF05C0E5FF06C00C
:10223000E5FF020EE56EF0EC18F0006EF3CF01F052
:10224000E12A040E015C02E1000E005C02E3006A78
:10225000016A8DEC06F00150E56E0050E56E000E4F
:10226000E56E200EE56E61EC16F0026EF3CF03F022
:10227000040EE126000E056E800E046E800E066EC2
:10228000200EE56E0650E56E0550E56E0450E56ED5
:10229000030EE56E0350E56E0250E56EA00EE56E8E
:1022A00093EC11F0080EE12601011BA31ED0020ED3
:1022B000E56E000EE56E200EE56ED60EE56EFDECC9
:1022C00016F0040EE126000E036E800E026E800EE4
:1022D000046E200EE56E0450E56E0350E56E02506C
:1022E000E56EFDEC16F0040EE126002AD8B0012AB6
:1022F0000150E56E0050E56E020EE56EB5EC18F08B
:10230000030EE126E4CF06F0E4CF05F0E4CF04F0BD
:10231000E4CF03F0E4CF02F0E4CF01F0E4CF00F02B
:10232000E4CFD9FF1200D9CFE5FFE1CFD9FF00C03C
:10233000E5FF01C0E5FF02C0E5FF03C0E5FF04C003
:10234000E5FF05C0E5FF06C0E5FF07C0E5FF020E9B
:10235000DBCF00F0030EDBCF01F0040EDBCF02F089
:10236000050EDBCF03F0060EDBCF04F0070EDBCF4C
:1023700005F0080EDBCF06F0090EDBCF07F073EC9B
:102380001AF003A003D0020EC86E02D0090EC86E68
:1023900028EC1CF00050E56E04EC1CF0E12A03A2CE
:1023A00008D00250006E036A0050E56E04EC1CF089
:1023B000E12A0150E56E04EC1CF0E12A04C000F0B3
:1023C00005C001F006C002F007C003F003C004F02E
:1023D0000306045013E000C0E9FF01C0F3FF025000
:1023E000AFEC1BF0046E002AD8B0012AD8B0022A44
:1023F0000450E56E04EC1CF0E12AE8D710EC1CF068
:10240000E86AE4CF07F0E4CF06F0E4CF05F0E4CFCC
:1024100004F0E4CF03F0E4CF02F0E4CF01F0E4CF26
:1024200000F0E4CFD9FF1200D9CFE5FFE1CFD9FF0B
:1024300000C0E5FF01C0E5FF02C0E5FF03C0E5FF06
:1024400004C0E5FF05C0E5FF06C0E5FF07C0E5FFE6
:10245000020EDBCF00F0030EDBCF01F0040EDBCF6A
:1024600002F0050EDBCF03F0D88001AED890046AED
:102470000436045007E0011C066E001C056E054A78
:10248000062A04D000C005F001C006F005C000F027
:1024900006C001F0D88003AED890056A0536055015
:1024A00007E0031C076E021C066E064A072A04D0CA
:1024B00002C006F003C007F00750E56E0650E56E57
:1024C0000150E56E0050E56E66EC15F0006EF3CF3E
:1024D00001F0040EE1260550041A04500AE0011C24
:1024E000036E001C026E024A032A03C0F3FF02506F
:1024F00003D001C0F3FF0050E4CF07F0E4CF06F0B3
:10250000E4CF05F0E4CF04F0E4CF03F0E4CF02F031
:10251000E4CF01F0E4CF00F0E4CFD9FF1200D9CF2F
:10252000E5FFE1CFD9FF00C0E5FF01C0E5FF02C034
:10253000E5FF03C0E5FF04C0E5FF020EDBCF00F0BE
:10254000030EDBCF01F0040EDBCF02F0050EDBCF74
:1025500003F0060EDBCF04F073EC1AF0090EC86E20
:1025600028EC1CF0C60EE56E04EC1CF0E12A000E0F
:10257000E56E04EC1CF0E12AFE0EE56E04EC1CF0A6
:10258000E12A0150400DF3CF01F0800E01260150E9
:1025900000260050E56E04EC1CF0E12A02C000F0B9
:1025A00003C001F004C002F000C0E9FF01C0F3FF66
:1025B0000250AFEC1BF0036E03500BE0002AD8B0C2
:1025C000012AD8B0022A0350E56E04EC1CF0E12A7F
:1025D000EBD7FF0EE56E04EC1CF0E12A10EC1CF0CA
:1025E000000EE56E0A0EE56EECEC0FF0020EE12631
:1025F000E4CF04F0E4CF03F0E4CF02F0E4CF01F045
:10260000E4CF00F0E4CFD9FF1200D9CFE5FFE1CF4E
:10261000D9FF00C0E5FF01C0E5FF02C0E5FF03C030
:10262000E5FF000EE56E000EE56E000EE56E0A0E8B
:10263000E56E0001C851E56E0001C751E56E00016D
:10264000C651E56E0001C551E56E7AEC10F0006EE2
:10265000F3CF01F0F4CF02F0E9CF03F0080EE1264A
:102660000350E56E0250E56E0150E56E0050E56ED8
:10267000000EE56E000EE56E000EE56E920EE56E44
:1026800000EC0BF0006EF3CF01F0F4CF02F0E9CFD5
:1026900003F0080EE126000EE56E000EE56E000E5A
:1026A000E56E640EE56E0350E56E0250E56E015076
:1026B000E56E0050E56E7AEC10F0006EF3CF01F09D
:1026C000F4CF02F0E9CF03F0080EE126005000013C
:1026D000F56F01500001F66FE4CF03F0E4CF02F094
:1026E000E4CF01F0E4CF00F0E4CFD9FF1200D9CF5E
:1026F000E5FFE1CFD9FF00C0E5FF01C0E5FF02C063
:10270000E5FF03C0E5FF000EE56E040EE56E000177
:10271000F251E56E0001F151E56E14EC12F0006E1D
:10272000F3CF01F0040EE1260001F1510026000173
:10273000F25101220150E56E0050E56E000EE56E8B
:102740000C0EE56E61EC16F0026EF3CF03F0040E92
:10275000E126D8900330016E0230006ED89001322D
:102760000032026A036A0001BC51035C0BE1000104
:10277000BB51025C07E10001BA51015C03E10001B9
:10278000B951005C0DE200500001B95F0150000139
:10279000BA5B02500001BB5B03500001BC5B08D078
:1027A0000001B96B0001BA6B0001BB6B0001BC6B8F
:1027B000E4CF03F0E4CF02F0E4CF01F0E4CF00F087
:1027C000E4CFD9FF1200D9CFE5FFE1CFD9FF00C098
:1027D000E5FF01C0E5FF02C0E5FF03C0E5FF04C05F
:1027E000E5FF05C0E5FF06C0E5FF07C0E5FF08C03F
:1027F000E5FF09C0E5FF020EDBCF00F0030EDBCFE3
:1028000001F0040EDBCF02F0050EDBCF03F0060E65
:10281000DBCF04F0070EDBCF05F000C006F001C0EF
:1028200007F002C008F003C0E9FF04C0F3FF055041
:10283000AFEC1BF0096E032AD8B0042AD8B0052AE1
:1028400009C0E5FF06C0E9FF07C0F3FF08504AECE6
:102850001CF0062AD8B0072AD8B0082A0950E3E1AC
:1028600002C0F4FF01C0F3FF0050E4CF09F0E4CF51
:1028700008F0E4CF07F0E4CF06F0E4CF05F0E4CFB2
:1028800004F0E4CF03F0E4CF02F0E4CF01F0E4CFB2
:1028900000F0E4CFD9FF1200D9CFE5FFE1CFD9FF97
:1028A00000C0E5FF01C0E5FF02C0E5FF03C0E5FF92
:1028B00004C0E5FF05C0E5FF06C0E5FF07C0E5FF72
:1028C00008C0E5FF09C0E5FF0AC0E5FF0BC0E5FF52
:1028D000020EDBCF00F00050E56EF0EC18F0016E58
:1028E000F3CF02F0E12A036A046A002A002A0050AA
:1028F000E56EF0EC18F0006EF3CF05F0E12A066A01
:10290000076A05500B6E00500A6E086A096A085083
:102910000112095002120A5003120B50041204C093
:10292000E9FF03C0F4FF02C0F3FF0150E4CF0BF056
:10293000E4CF0AF0E4CF09F0E4CF08F0E4CF07F0E9
:10294000E4CF06F0E4CF05F0E4CF04F0E4CF03F0E9
:10295000E4CF02F0E4CF01F0E4CF00F0E4CFD9FF00
:102960001200D9CFE5FFE1CFD9FF00C0E5FF01C0DC
:10297000E5FF02C0E5FF03C0E5FF04C0E5FF05C0B9
:10298000E5FF06C0E5FF020EDBCF00F0030EDBCF54
:1029900001F0040EDBCF02F0050EDBCF03F0046A7A
:1029A000056A0344010B066E06B011D002500226E0
:1029B00003360350015C02E10250005C04E2D8904F
:1029C0000332023204D0052A05C004F0EAD70350CE
:1029D000015C02E10250005C04E30250005E03501F
:1029E000015AD8900332023204C005F004060550A3
:1029F000EEE101C0F3FF0050E4CF06F0E4CF05F0B4
:102A0000E4CF04F0E4CF03F0E4CF02F0E4CF01F030
:102A1000E4CF00F0E4CFD9FF1200D9CFE5FFE1CF3A
:102A2000D9FFE80E0101066F030E0101076FE80EE2
:102A30000101086F030E0101096F0001B96B00016C
:102A4000BA6BE80E0001BB6F030E0001BC6F000102
:102A5000C56B0001C66B0001C76B0001C86B0001AC
:102A6000FB6B0001FC6B0001FD6B0001FE6B000EB7
:102A7000E56E000EE56E020EE56EB5EC18F0030E85
:102A8000E12601010751E56E01010651E56E060ED2
:102A9000E56EB5EC18F0030EE12601010951E56E73
:102AA00001010851E56E080EE56EB5EC18F0030E55
:102AB000E126000EE56E080EE56E0C0EE56EB5EC37
:102AC00018F0030EE126E4CFD9FF1200D9CFE5FFBD
:102AD000E1CFD9FF00C0E5FF01C0E5FF02C0E5FF7F
:102AE00003C0E5FF04C0E5FF05C0E5FF06C0E5FF44
:102AF00007C0E5FF020EDBCF00F0030EDBCF01F0D5
:102B0000040EDBCF02F0050EDBCF03F0046A056A8A
:102B1000100E066E0144010B076E010E07160050E1
:102B2000002601360450042605360750D8A4048038
:102B30000350055C02E10250045C05E30250045EB0
:102B40000350055A0080062EE5D701C0F3FF005060
:102B5000E4CF07F0E4CF06F0E4CF05F0E4CF04F0D3
:102B6000E4CF03F0E4CF02F0E4CF01F0E4CF00F0D3
:102B7000E4CFD9FF1200D9CFE5FFE1CFD9FF00C0E4
:102B8000E5FF01C0E5FF02C0E5FF020EDBCF00F06C
:102B900000380F0B016E300E01263A0E015C02E385
:102BA000070E012601500001E86F0F0E0014016EA0
:102BB000300E01263A0E015C02E3070E0126015099
:102BC0000001E96F0001EA69000E016EE80E006E77
:102BD000800E026E030EE56E0250E56E0150E56E4A
:102BE0000050E56E000EE56E000EE56E000EE56E1F
:102BF000C60EE56E93EC11F0080EE126000EE56EB0
:102C00000A0EE56EECEC0FF0020EE126E4CF02F0C6
:102C1000E4CF01F0E4CF00F0E4CFD9FF1200D9CF28
:102C2000E5FFE1CFD9FF00C0E5FF01C0E5FF02C02D
:102C3000E5FF03C0E5FF04C0E5FF05C0E5FF06C0F2
:102C4000E5FF020EDBCF00F0030EDBCF01F0040E38
:102C5000DBCF02F0050EDBCF03F0060EDBCF04F076
:102C60000150056E0250066E0650E56E0550E56E89
:102C70000050E56EB5EC18F0030EE126002A002A9C
:102C80000350016E0450026E036A046A0250E56E3E
:102C90000150E56E0050E56EB5EC18F0030EE1262C
:102CA000E4CF06F0E4CF05F0E4CF04F0E4CF03F086
:102CB000E4CF02F0E4CF01F0E4CF00F0E4CFD9FF9D
:102CC0001200D9CFE5FFE1CFD9FF00C0E5FF01C079
:102CD000E5FF02C0E5FF03C0E5FF020EDBCF00F019
:102CE000030EDBCF01F0040EDBCF02F0050EDBCFCD
:102CF00003F000500101126F0150136F02500101E7
:102D0000146F0350156F0101125101011403F3CF29
:102D100000F0F4CF01F000500101166F0150176F61
:102D20000101125101011503F3CF00F0010113510C
:102D300001011403F3CF01F00150002601011751E6
:102D400000260050176F17C1F3FF1651E4CF03F0B0
:102D5000E4CF02F0E4CF01F0E4CF00F0E4CFD9FFFC
:102D60001200A80EF66E380EF76E000EF86E09000F
:102D7000F550056E0900F550066E055002E106504B
:102D80003BE00900F550006E0900F550016E0900A6
:102D9000F550026E09000900F550E96E0900F55082
:102DA000EA6E090009000900F550036E0900F550AC
:102DB000046E09000900F6CF07F0F7CF08F0F8CF4E
:102DC00009F000C0F6FF01C0F7FF02C0F8FF035092
:102DD00002E1045007E00900F550EE6E0306F8E248
:102DE0000406F9D707C0F6FF08C0F7FF09C0F8FFCF
:102DF0000506C4E20606C5D71200D9CFE5FFE1CF2C
:102E0000D9FF00C0E5FF01C0E5FF02C0E5FF03C038
:102E1000E5FF04C0E5FF05C0E5FF020EDBCF00F0D3
:102E2000030EDBCF01F0040EDBCF02F0050EDBCF8B
:102E300003F0046A0350045C14E200C0E9FF01C01F
:102E4000F3FF0250AFEC1BF0056E002AD8B0012A48
:102E5000D8B0022A0550E56E9DEC1BF0E12A042A49
:102E6000E9D7E4CF05F0E4CF04F0E4CF03F0E4CFFA
:102E700002F0E4CF01F0E4CF00F0E4CFD9FF12007C
:102E8000D9CFE5FFE1CFD9FF00C0E5FFCFEC1BF0C4
:102E9000006E005031E040EC1CF0006E0050520A11
:102EA00029E00050630A1AE00050640A1BE0005059
:102EB0006D0A07E00050720A0DE00050740A17E036
:102EC0001BD00101182B040E0101185D15E301014F
:102ED000186B12D0010E01011B6F0ED0030E010101
:102EE0001B6F0AD001011B6BCCEC09F005D00AEC7A
:102EF0000CF002D00DEC15F0E4CF00F0E4CFD9FFD8
:102F00001200D9CFE5FFE1CFD9FF00C0E5FF01C036
:102F1000E5FF02C0E5FF03C0E5FFFDEC17F0006E22
:102F2000F3CF01F001010051005C026E010101517B
:102F30000158036E000E035C02E1330E025C14E3E1
:102F400000C000F101C001F10001C52B02E3000146
:102F5000C62B02E30001C72B02E30001C82B0101CD
:102F6000022B02E30101032BE4CF03F0E4CF02F0D4
:102F7000E4CF01F0E4CF00F0E4CFD9FF1200D9CFC5
:102F8000E5FFE1CFD9FF00C0E5FF01C0E5FF02C0CA
:102F9000E5FF03C0E5FFD5EC19F0006EF3CF01F0BB
:102FA000F4CF02F0E9CF03F0000EE56E0F0EE56EF0
:102FB000420EE56E400EE56E0350E56E0250E56E82
:102FC0000150E56E0050E56E7AEC10F0006EF3CF24
:102FD00001F0F4CF02F0E9CF03F0080EE12601C0C2
:102FE000F3FF0050E4CF03F0E4CF02F0E4CF01F0B0
:102FF000E4CF00F0E4CFD9FF1200D9CFE5FFE1CF55
:10300000D9FF00C0E5FF01C0E5FF02C0E5FF03C036
:10301000E5FFD5EC19F0006EF3CF01F0F4CF02F02C
:10302000E9CF03F0000EE56E000EE56E030EE56ECF
:10303000E80EE56E0350E56E0250E56E0150E56E58
:103040000050E56E7AEC10F0006EF3CF01F0F4CF93
:1030500002F0E9CF03F0080EE12601C0F3FF0050B3
:10306000E4CF03F0E4CF02F0E4CF01F0E4CF00F0CE
:10307000E4CFD9FF1200D9CFE5FFE1CFD9FF00C0DF
:10308000E5FF01C0E5FF02C0E5FF020EDBCF00F067
:1030900000500001ED6F0001EE69000E016EED0EB3
:1030A000006E800E026E020EE56E0250E56E01505B
:1030B000E56E0050E56E000EE56E000EE56E000E4A
:1030C000E56EC60EE56E93EC11F0080EE126000EDB
:1030D000E56E0A0EE56EECEC0FF0020EE126E4CF91
:1030E00002F0E4CF01F0E4CF00F0E4CFD9FF12000A
:1030F000D9CFE5FFE1CFD9FF00C0E5FF01C0E5FF73
:1031000002C0E5FFFE0E0001E56F010E0001E66F53
:103110000001E769000E016EE50E006E800E026E82
:10312000030EE56E0250E56E0150E56E0050E56E4F
:10313000000EE56E000EE56E000EE56EC60EE56E45
:1031400093EC11F0080EE126000EE56E0A0EE56E16
:10315000ECEC0FF0020EE126E4CF02F0E4CF01F038
:10316000E4CF00F0E4CFD9FF1200D9CFE5FFE1CFE3
:10317000D9FF00C0E5FF01C0E5FF02C0E5FF020E78
:10318000DBCF00F0030EDBCF01F0040EDBCF02F04B
:10319000A69EA69CA684F29E00C0A9FF0150A86E20
:1031A000550EA76EAA0EA76EA682A6B2FED700285D
:1031B000A96E0250016E026A0150A86E550EA76EEC
:1031C000AA0EA76EA682A6B2FED7A694F28EE4CF70
:1031D00002F0E4CF01F0E4CF00F0E4CFD9FF120019
:1031E000D9CFE5FFE1CFD9FF00C0E5FF01C0E5FF82
:1031F00002C0E5FF03C0E5FF04C0E5FF05C0E5FF31
:10320000020EDBCF00F0A69CA69E00C0A9FFA68000
:10321000A8CF01F0026A0028A96EA680A8CF00F00E
:10322000036A0050056E046A045001120550021230
:1032300002C0F3FF0150E4CF05F0E4CF04F0E4CF87
:1032400003F0E4CF02F0E4CF01F0E4CF00F0E4CFEC
:10325000D9FF1200D9CFE5FFE1CFD9FF00C0E5FFCC
:1032600001C0E5FF02C0E5FF03C0E5FF020EDBCFB2
:1032700000F0030EDBCF01F0040EDBCF02F000C044
:10328000E9FF01C0F3FF0250AFEC1BF0036E0350E7
:1032900010E0ACA2FED700C0E9FF01C0F3FF02506E
:1032A000AFEC1BF0AD6E002AD8B0012AD8B0022ACC
:1032B000E6D7E4CF03F0E4CF02F0E4CF01F0E4CFAF
:1032C00000F0E4CFD9FF1200D9CFE5FFE1CFD9FF5D
:1032D00000C0E5FF01C0E5FF02C0E5FF03C0E5FF58
:1032E000020EDBCF00F0030EDBCF01F0026A036AAF
:1032F00001BE0CD0D89001360150005C03E2D8909A
:10330000013204D0032A03C002F0F2D70150005C5E
:1033100002E30150005ED890013202C003F00206C1
:103320000350F4E10050E4CF03F0E4CF02F0E4CF27
:1033300001F0E4CF00F0E4CFD9FF1200D9CFE5FFD0
:10334000E1CFD9FF00C0E5FF01C0E5FF02C0E5FF06
:1033500003C0E5FF04C0E5FF020EDBCF00F0030E63
:10336000DBCF01F0026A080E036E800E0014046EBB
:10337000D8900036D89002360450D8A4028001506C
:10338000025C03E30150025E0080032EEED7005082
:10339000E4CF04F0E4CF03F0E4CF02F0E4CF01F097
:1033A000E4CF00F0E4CFD9FF120000C0E5FF01C078
:1033B000E5FF02C0E5FF03C0E5FF04C0E5FF05C06F
:1033C000E5FFB2CF00F0B3CF01F0EFC002F0F0C0E4
:1033D00003F0B2CF04F0B3CF05F00150055C02E179
:1033E0000050045C04E2EFC002F0F0C003F003C040
:1033F000E9FF02C0F4FF05C0F3FF0450E4CF05F07D
:10340000E4CF04F0E4CF03F0E4CF02F0E4CF01F026
:10341000E4CF00F01200E8CFE5FFD8CFE5FFE0CF22
:10342000E5FFF3CFE5FFF4CFE5FFE9CFE5FFEACF16
:10343000E5FFFACFE5FFFBCFE5FFD9CFE5FFE1CF11
:10344000D9FFA1A203D0F8EC1BF0A192F2A203D005
:1034500081EC17F0F292E4CFD9FFE4CFFBFFE4CF89
:10346000FAFFE4CFEAFFE4CFE9FFE4CFF4FFE4CFD3
:10347000F3FFE4CFE0FFE4CFD8FFE4CFE8FF100094
:10348000D9CFE5FFE1CFD9FF00C0E5FF01C0E5FFDF
:1034900002C0E5FF03C0E5FF020EDBCF00F00044F1
:1034A000E844FC0B016E030E0110C26EC2B2FED7DF
:1034B000C4CF00F0016A0050036E026AC3CF00F06F
:1034C000016A005002260150032203C0F3FF02509C
:1034D000E4CF03F0E4CF02F0E4CF01F0E4CF00F05A
:1034E000E4CFD9FF1200D9CFE5FFE1CFD9FF00C06B
:1034F000E5FF01C0E5FF02C0E5FFFF0E006E1F0EF5
:10350000C514016E026AC7B4022A025001120150AA
:1035100003E000060050F3E100C001F0005002E1BA
:1035200049EC1BF00150D880E866D890016A01365A
:103530000150E4CF02F0E4CF01F0E4CF00F0E4CF9B
:10354000D9FF1200D9CFE5FFE1CFD9FF000EE56E1C
:10355000200EE56EDA0EE56E000EE56E000EE56EED
:103560008FEC12F0050EE126000EE56E200EE56EE2
:10357000E00EE56E010EE56E000EE56E8FEC12F0CA
:10358000050EE126070EE56ED00EE56EECEC0FF0B1
:10359000020EE126E4CFD9FF1200D9CFE5FFE1CF3B
:1035A000D9FF00C0E5FF01C0E5FF020EDBCF00F050
:1035B000030EDBCF01F0A69EA69CA684F29E01C05E
:1035C000A8FF00C0A9FF550EA76EAA0EA76EA6827F
:1035D000A6B2FED7A694F28EE4CF01F0E4CF00F0BD
:1035E000E4CFD9FF1200D9CFE5FFE1CFD9FF00C06A
:1035F000E5FF01C0E5FF020EDBCF00F073EC1AF02F
:10360000C58673EC1AF0C9CF01F073EC1AF00050C4
:1036100002E0C59A01D0C58AC5880150E4CF01F007
:10362000E4CF00F0E4CFD9FF1200D9CFE5FFE1CF1E
:10363000D9FF01011AA110D0000EE56E200EE56E33
:10364000C40EE56E010EE56E000EE56E8FEC12F015
:10365000050EE126818E01D0819EE4CFD9FF1200B4
:10366000D9CFE5FFE1CFD9FF00C0E5FF01C0E5FFFD
:103670001F0EC514006E016AC7B4012A0150001262
:103680000050F6E1E4CF01F0E4CF00F0E4CFD9FF41
:103690001200D9CFE5FFE1CFD9FF818AC69A94966F
:1036A000828682B803D082968286FBD794988298CD
:1036B000828894869488C68AE4CFD9FF1200D9CF35
:1036C000E5FFE1CFD9FF200EAC6E900EAB6E0C0E75
:1036D000AF6E000EE56E010EE56EECEC0FF0020E23
:1036E000E126E4CFD9FF1200D9CFE5FFE1CFD9FF22
:1036F0003F0EC716280EC66EC56A090EC86E9486A0
:1037000094889E96A19649EC1BF0819AE4CFD9FF4C
:103710001200D9CFE5FFE1CFD9FF00C0E5FF020ECF
:10372000DBCF00F0A69CA69E00C0A9FFA680A850F3
:10373000E4CF00F0E4CFD9FF1200D9CFE5FFE1CF0D
:10374000D9FF00C0E5FF020EDBCF00F0ACA2FED730
:1037500000C0ADFFE4CF00F0E4CFD9FF1200E8AE27
:1037600004D0F3CFEAFFEE501200E8BC08D0E9CF56
:10377000F6FFF3CFF7FFF86E0900F55012001200C4
:10378000D9CFE5FFE1CFD9FF810EB16EB36AB26A3E
:103790000001EF6B0001F06BE4CFD9FF1200D9CF2D
:1037A000E5FFE1CFD9FF00C0E5FF006A9EBA002A1D
:1037B0000050E4CF00F0E4CFD9FF1200D9CFE5FFED
:1037C000E1CFD9FF010EC26E050EC16E940EC06E20
:1037D000E4CFD9FF1200D9CFE5FFE1CFD9FFB36A1B
:1037E000B26A0001EF6B0001F06BE4CFD9FF120069
:1037F000D9CFE5FFE1CFD9FF0001EF2B02E30001B4
:10380000F02BE4CFD9FF1200D9CFE5FFE1CFD9FFEC
:10381000020EDBCFC9FF73EC1AF0E4CFD9FF120020
:10382000D9CFE5FFE1CFD9FF73EC1AF0C584C5B459
:10383000FED7E4CFD9FF1200D9CFE5FFE1CFD9FF02
:1038400073EC1AF0C582C5B2FED7E4CFD9FF1200DF
:10385000D9CFE5FFE1CFD9FF73EC1AF0C580C5B031
:10386000FED7E4CFD9FF120012EEFFF022EEFFF0F8
:10387000F86AA68EA69CB1EC16F0B3EC03F0FFD765
:10388000D9CFE5FFE1CFD9FF9EAAFED7AE50E4CF56
:10389000D9FF1200E8AE05D0F3CFEAFFE4CFEEFF88
:1038A0001200E8AC120012000100B63800001E0140
:0838B00000000100000000000F
:00000001FF
